:1018650090FFFE120538ECF0A3EDF090FFFD120598
:1018750038EBF0A3EAF0A3E9F0850883850982E057
:10188500F9A3E0FAA3E09003ADC9F0A3EAF0A3E958
:10189500F090000312055CE0FFA3E09003B2CFF0E7
:1018A500A3EFF0E49003B0F0A3F0850883850982E7
:1018B500E0FBA3E0FAA3E0F912011CF5999003B24D
:1018C500E0FEA3E0FFC39003B1E09FEE6480F890D3
:0E18D50003B0E064809840E5900005020538FD
:1016DD0057656C636F6D6520746F204D43553132C6
:1016ED00332E434F4D200D0A005461736B31206929
:1016FD00732072756E6E696E6721204C4544313DC5
:10170D004F4E200D0A0075436F7349495F56657240
:10171D00005461736B322069732072756E6E696E41
:10172D006721204C4544323D4F4E200D0A00546137
:10173D00736B332069732072756E6E696E6721202D
:10174D004C4544313D4F4646204C4544323D4F4675
:05175D0046200D0A000A
:1013160090039FEEF0A3EFF0A3EBF0A3EAF0A3E9AE
:01132600F0D6
:10132700E4A3F090039FE0FAA3E0FB7C007D0AFFB3
:10133700AE02120196ED2430FF9003A4E024A5F538
:1013470082E43403F583EFF07C007D0AAF03AE023D
:1013570012019690039FEEF0A3EFF04E600A900300
:10136700A4E004F0E0B405BB9003A4E0FFD394002D
:10137700402874A52FF582E43403F583E0FF90033A
:10138700A1E0FBA3E475F001120201A9F0FAEF1244
:1013970001629003A4E014F080CE9003A4E024A59A
:1013A700F582E43403F583E0FF9003A1E0FBA3E4B7
:1013B70075F001120201A9F0FAEF1201629003A180
:1013C700E0FBA3E0FAA3E0F9740D1201629003A217
:1013D700E475F0011201EB9003A1E0FBA3E0FAA38F
:0713E700E0F9740A02016243
:1013EE00120ACA121BC090FFFF1205387402F07B5E
:1013FE00017A02796B90FFFD120538EBF0A3EAF04B
:10140E00A3E9F07B007A00790090FFFD120538EB1E
:10141E00F0A3EAF0A3E9F07BFF7A12792E120E8C7C
:10142E0090FFFF1205387403F07B017A0279CF909A
:10143E00FFFD120538EBF0A3EAF0A3E9F07B007A8A
:10144E0000790090FFFD120538EBF0A3EAF0A3E956
:10145E00F07BFF7A197950120E8C90FFFF1205382F
:10146E007404F07B017A03793390FFFD120538EB9B
:10147E00F0A3EAF0A3E9F07B007A00790090FFFD7B
:10148E00120538EBF0A3EAF0A3E9F07BFF7A1879A6
:07149E00E3120E8C0217E5BA
:10122E0090FFFD120538EBF0A3EAF0A3E9F090FF72
:04123E00BF1205389E
:10124200850883850982A982AA83A801AC027D014F
:101252007BFF7A1679DD7E007F191200F67B019002
:10126200001912055CA982AA83A801AC02AD037B16
:10127200FF7A1679F67E007F1D1200F67B01900040
:101282003612055CA982AA83A801AC02AD037BFFDA
:101292007A1779137E007F0B1200F6900041120537
:1012A2005CE0FBA3E0FAA3E0F990004112055CEBDD
:1012B200F0A3EAF0A3E9F07C007D197B01850883A5
:1012C200850982A982AA831218651200037B017A1A
:1012D2000379971213167C007D0B7B019000361266
:1012E200055CA982AA831218657C007D087B017ABD
:1012F200037997121865C2957C007D1D7B019000D1
:101302001912055CA982AA831218657E007F6412F5
:04131200176280E2FC
:1019500090FFFD120538EBF0A3EAF0A3E9F090FF49
:04196000E312053851
:10196400850883850982A982AA83A801AC027D0126
:101974007BFF7A17791E7E007F1D1200F690001DF2
:1019840012055CE0FBA3E0FAA3E0F990001D120548
:101994005CEBF0A3EAF0A3E9F0C2967C007D1D7B2A
:1019A40001850883850982A982AA831218657E00AD
:0719B4007F6412176280E25C
:1018E30090FFFD120538EBF0A3EAF0A3E9F090FFB7
:0418F300D9120538C9
:1018F700850883850982A982AA83A801AC027D0194
:101907007BFF7A17793B7E007F271200F69000272E
:1019170012055CE0FBA3E0FAA3E0F99000271205AB
:101927005CEBF0A3EAF0A3E9F0D295D2967C007DB8
:10193700277B01850883850982A982AA83121865F6
:091947007E007F3212176280E07D
:10111E004801FD0102040810204080610000D20049
:10112E0000010002000100030001000200010004A2
:10113E000001000200010003000100020001000591
:10114E000001000200010003000100020001000482
:10115E000001000200010003000100020001000670
:10116E000001000200010003000100020001000462
:10117E000001000200010003000100020001000551
:10118E000001000200010003000100020001000442
:10119E00000100020001000300010002000100072F
:1011AE000001000200010003000100020001000422
:1011BE000001000200010003000100020001000511
:1011CE000001000200010003000100020001000402
:1011DE0000010002000100030001000200010006F0
:1011EE0000010002000100030001000200010004E2
:1011FE0000010002000100030001000200010005D1
:10120E0000010002000100030001000200010004C1
:0F121E00000100020001000300010002000100B6
:060ACA0090FFF512053853
:100AD0001200089001D212042300000000E47810F4
:100AE000F6780CF6781DF6780BF6781912040A00E1
:100AF000000000781512040A00000000E4780AF6ED
:100B0000850883850982A3A304F0A37402F0A3746B
:100B100069F0850883850982E4F0A3F08508838560
:100B20000982E0FEA3E0C39402EE940050278508FA
:100B300083850982A3A3E0FBA3E475F001120201FF
:100B4000A9F0FAE412016285088385098275F00133
:100B50001201EB80C7E4781EF608F67811F608F665
:100B600008F6780DF608F608F6F9900000C9F0A32B
:100B7000F0A3E9F0850883850982E4F0A3F08508F5
:100B800083850982E0FEA3E0FFC3940DEE9400503C
:100B9000279001D675F003EF120454EE75F003A40C
:100BA0002583F583E4F0A3F0A3F08508838509820B
:100BB00075F0011201EB80C67B017A007903900089
:100BC0000512055CEBF0A3EAF0A3E9F07B017A00E3
:100BD000791490000812055CEBF0A3EAF0A3E9F0A9
:100BE000850883850982E4F0A3F08508838509825E
:100BF000E0FEA3E0C3940BEE940050539000081263
:100C0000055CE0FBA3E0FAA3E0F9C003C002C00169
:100C100090000512055CE0FBA3E0FAA3E0F9900068
:100C2000031204DF90000512055CA3E475F01112B5
:100C300001EB90000812055CA3E475F0111201EBC2
:100C4000850883850982E475F0011201EB809B7BA6
:100C5000007A007900C003C002C0019000051205AF
:100C60005CE0FBA3E0FAA3E0F99000031204DF903C
:100C700000CF7401F0A37400F0A37403F090FFFFA1
:100C8000120538740CF07B017A02790590FFFD1291
:100C90000538EBF0A3EAF0A3E9F07B007A007900D5
:100CA00090FFFD120538EBF0A3EAF0A3E9F07BFF1B
:0A0CB0007A1A7973120E8C120009F3
:060CBA0090000B0205385A
:0E000E00C2AF7810E6C394FF500106D2AF22B5
:10165300C2AF7810E6D394004001167810E6707795
:10166300780CE67072780AE624D2F582E43400F549
:1016730083E07814F6E6FF2469F582E43402F58307
:10168300E024D2F582E43400F583E0FEEF33333314
:1016930054F8FFEE2FFF781FF618E66F603908E65F
:1016A30075F003A424D6F582E43401F583E0FBA3AB
:1016B300E0FAA3E07811A60308A60208F67815124B
:1016C30003E6EF2401FFE43EFEE43DFDE43CFC7849
:0A16D300151203F2121BE4D2AF223D
:0617E50090FFFE12053822
:1017EB00780BE6706F18E624D2F582E43400F583AB
:1017FB00E0850883850982F0E0FF2469F582E434F3
:10180B0002F583E024D2F582E43400F583E0850809
:10181B0083850982A3F0EF33333354F8FF850883B4
:10182B00850982A3E02F781FF618F675F003A42420
:10183B00D6F582E43401F583E0FBA3E0FAA3E0786C
:10184B0011A60308A60208F6780DA60308A602083F
:04185B00F6121A2146
:06185F00900002020538B2
:06100C0090FFFD12053803
:1010120012001CC2AF9001D2E0FCA3E0FDA3E0FEEF
:10102200A3E02401FFE43EFEE43DFDE43CFC90012C
:10103200D21203FED2AF900000E0F9A3E0FAA3E0DF
:10104200850883850982C9F0A3EAF0A3E9F085083F
:1010520083850982E0FBA3E0FAA3E0F990000C1279
:101062000135640C7003021118C2AF90000912021C
:101072001745F0607A850883850982E0FBA3E0FAD0
:10108200A3E0F990000974FFF5F012024F45F070E9
:101092005E90000B12013520E33D900010120135E5
:1010A200780A46F690000E1201352469F582E4347E
:1010B20002F583C083C082E0FF850883850982E050
:1010C200FBA3E0FAA3E0F990000F120135FEEF4E08
:1010D200D082D083F08018850883850982E0FBA343
:1010E200E0FAA3E0F9900009E475F00112029C8590
:1010F2000883850982E0FBA3E0FAA3E0F9900003EC
:101102001204AF850883850982EBF0A3EAF0A3E914
:06111200F0D2AF02105004
:06111800900003020538FF
:050003007E007FFB22DE
:0615370090FFFF120538D1
:10153D00C2AF7810E6707B780CE67076780AE624F8
:10154D00D2F582E43400F583E0850883850982F0C5
:10155D00E0FF2469F582E43402F583E024D2F582BC
:10156D00E43400F583E0FEEF33333354F8FFEE2F10
:10157D00FF781FF618E66F603908E675F003A424AE
:10158D00D6F582E43401F583E0FBA3E0FAA3E0781D
:10159D0011A60308A60208F678151203E6EF24013A
:1015AD00FFE43EFEE43DFDE43CFC78151203F2122F
:0415BD0019BBD2AFD5
:0615C10090000102053854
:101A730090FFFD120538EBF0A3EAF0A3E9F0850827
:101A830083850982E0F9A3E0FAA3E0850883850949
:101A930082C9F0A3EAF0A3E9F0C2AF78191203E612
:101AA300EF2401FFE43EFEE43DFDE43CFC78191223
:091AB30003F2D2AF12001D80E025
:1005AB0090FFFD120538EBF0A3EAF0A3E9F090FF02
:0C05BB00FF120538EFF090FFFD1205382C
:1005C700C2AF9000CFE0F9A3E0FAA3E085088385E6
:1005D7000982C9F0A3EAF0A3E9F0850883850982B7
:1005E700E0FBA3E0FAA3E04A4B700302085D85082D
:1005F70083850982E0FBA3E0FAA3E0F990000312E8
:1006070004AF9000CFEBF0A3EAF0A3E9F0D2AF90EC
:10061700000412055CE0FBA3E0FAA3E0F9C003C005
:1006270002C001850883850982E0FBA3E0FAA3E005
:10063700F912046090000312055CE0FF85088385CA
:100647000982E0FBA3E0FAA3E0F990000CEF1201A6
:100657007490000BE4120174900009E4F5F01202A3
:100667009C90001012055CE0FBA3E0FAA3E0F99070
:10067700001012055CEBF0A3EAF0A3E9F090000C80
:1006870012055CE0FCA3E0FDA3E0FEA3E0FF900001
:100697000C12055C1203FE90000712055CE0FBA339
:1006A700E0FAA3E0F990000712055CEBF0A3EAF08B
:1006B700A3E9F090001312055CE0FEA3E0FF9000B1
:1006C7001312055CEEF0A3EFF090000A12055CE050
:1006D700FEA3E0FF90000A12055CEEF0A3EFF09096
:1006E700000312055CE0FF131313541FFE850883F4
:1006F700850982E0FBA3E0FAA3E0F990000EEE1271
:10070700017490000E12013524FDF582E43401F5E1
:1007170083E0900010120174EF540790000D12014E
:100727007490000D12013524FDF582E43401F58340
:10073700E090000F120174121B67850883850982F8
:10074700E0FBA3E0FAA3E0F9121B38C2AF850883E8
:10075700850982E0FBA3E0FAA3E0F9900003120504
:100767005CE075F003A424D6F582E43401F583EB4D
:10077700F0A3EAF0A3E9F0900000E0FBA3E0FAA3FE
:10078700E0F9C003C002C001850883850982E0FB48
:10079700A3E0FAA3E0F99000031204DF7B007A00DC
:1007A7007900C003C002C001850883850982E0FB88
:1007B700A3E0FAA3E0F99000061204DF900000E03E
:1007C700FBA3E0FAA3E04A4B6025850883850982ED
:1007D700E0FBA3E0FAA3E0F9C003C002C001900068
:1007E70000E0FBA3E0FAA3E0F99000061204DF851E
:1007F7000883850982E0F9A3E0FAA3E0900000C925
:10080700F0A3EAF0A3E9F0850883850982E0FBA35A
:10081700E0FAA3E0F9900010120135780A46F69045
:10082700000E1201352469F582E43402F583C08392
:10083700C082E0FF850883850982E0FBA3E0FAA375
:10084700E0F990000F120135FEEF4ED082D083F011
:0A085700D2AF7F008004D2AF7F46CD
:06086100900015020538AD
:1008670090FFFD120538EBF0A3EAF0A3E9F090FF43
:10087700FD12053890000612055CE0FBA3E0FAA321
:10088700E0F990000612055CEBF0A3EAF0A3E9F0AB
:1008970090000C12055CE0FEA3E0FF90000C12052F
:1008A7005CEEF0A3EFF090000912055CE0F9A3E01D
:1008B700FAA3E0850883850982C9F0A3EAF0A3E9D2
:1008C700F0850883850982E0FBA3E475F001120235
:1008D70001A9F0FA740F12016290000312055CA3DC
:1008E700A3E0FF850883850982E0FBA3E475F00197
:1008F700120201A9F0FAEF12016290000312055CDF
:10090700A3E0FAEAFF850883850982E0FBA3E47583
:10091700F001120201A9F0FAEF120162850883853E
:100927000982E0FBA3E475F001120201A9F0FA7451
:100937000A120162850883850982E0FBA3E475F04A
:1009470001120201A9F0FA740B120162850883856E
:100957000982E0FBA3E475F001120201A9F0FAE4B1
:10096700120162850883850982E0FBA3E475F00123
:10097700120201A9F0FAE41201628508838509824F
:10098700E0FBA3E475F001120201A9F0FAE41201F9
:1009970062850883850982E0FBA3E475F0011202F2
:1009A70001A9F0FAE412016290000612055CA3A304
:1009B700E0FF850883850982E0FBA3E475F0011257
:1009C7000201A9F0FAEF12016290000612055CA37A
:1009D700E0FAEAFF850883850982E0FBA3E475F066
:1009E70001120201A9F0FAEF120162850883850955
:1009F70082E0FBA3E475F001120201A9F0FA740189
:100A0700120162850883850982E0FBA3E475F00182
:100A1700120201A9F0FA740412016285088385099C
:100A270082E0FBA3E475F001120201A9F0FA740554
:100A3700120162850883850982E0FBA3E475F00152
:100A4700120201A9F0FA740612016285088385096A
:100A570082E0FBA3E475F001120201A9F0FA740722
:100A670012016290000912055CA3E0FAA3E0246476
:0C0A7700E43AFF850883850982E0FBA3B8
:100A8300E475F001120201A9F0FAEF12016290007D
:100A93000912055CA3A3E02464F9AF0185088385EB
:100AA3000982E0FBA3E475F001120201A9F0FAEF59
:100AB30012016290000912055CE0FBA3E0FAA3E0D7
:070AC300F990000E02053856
:0100080022D5
:0100090022D4
:101B380090FFFD120538EBF0A3EAF0A3E9F0850861
:101B480083850982E0F9A3E0FAA3E0850883850983
:0F1B580082C9F0A3EAF0A3E9F090000302053878
:01000A0022D3
:101B670090FFFD120538EBF0A3EAF0A3E9F0850832
:101B770083850982E0F9A3E0FAA3E0850883850954
:0F1B870082C9F0A3EAF0A3E9F090000302053849
:01001C0022C1
:01001D0022C0
:091BEE00758C70E4F58AD28C229A
:03000B00021ABC1A
:101ABC00C0E0C0F0C083C082C0D075D000C000C0F0
:101ACC0001C002C003C004C005C006C00712000E4E
:101ADC00121BEE12100C121653D007D006D005D0E4
:101AEC0004D003D002D001D000D0D0D082D083D08B
:041AFC00F0D0E03214
:030023000215C7FC
:1015C700C0E0C0F0C083C082C0D075D000C000C0EA
:1015D70001C002C003C004C005C006C00712000E48
:1015E700C2AF309942C2999003B1E004F0700690FF
:1015F70003B0E004F09003B2E0FEA3E0FF9003B075
:10160700E0FCA3E0FDC39FEE6480F8EC6480985093
:101617001B9003ADE0FBA3E0FAA3E0F98D828C8376
:10162700120135F5998005309802C298D2AF12168B
:1016370053D007D006D005D004D003D002D001D0B4
:0C16470000D0D0D082D083D0F0D0E032B0
:101BC000758921758C70E4F58AD28C758DFAC2AB5B
:101BD000D28E759850D2AC9003B0F0A3F0A3F0A3CE
:041BE000F0D2A92274
:100E8C0090FFFD120538EBF0A3EAF0A3E9F090FF18
:040E9C00FC12053807
:100EA00090000D12055CE0FED3940C40057F2A02F1
:100EB0001006C2AFEE75F003A424D6F582E4340127
:100EC000F583E0FBA3E0FAA3E04A4B6003021002C3
:100ED000FBFA790190000D12055CE075F003A42483
:100EE000D6F582E43401F583EBF0A3EAF0A3E9F050
:100EF000D2AF90FFFE120538E4F0A3F090000C1280
:100F0000055CE0FBA3E0FAA3E0F990FFFD120538D1
:100F1000EBF0A3EAF0A3E9F090000C12055CE0FB13
:100F2000A3E0FAA3E0F990FFFD120538EBF0A3EA85
:100F3000F0A3E9F090000C12055CE0FBA3E0FAA33B
:100F4000E0F9120867850883850982EBF0A3EAF0CF
:100F5000A3E9F090FFFE120538E4F0A3F0FBFAF9E4
:100F600090FFFD120538EBF0A3EAF0A3E9F090FF43
:100F7000FC1205381204230000000090FFFE120549
:100F800038E4F0A3F0FBFAF990FFFD120538EBF01E
:100F9000A3EAF0A3E9F090000E12055CE0FBA3E0E9
:100FA000FAA3E0F990001B12055CE0FF1205AB907C
:100FB000000312055CEFF090000312055CE0701274
:100FC000C2AF781D06D2AF780BE6B4012B121537ED
:100FD0008026C2AF7B007A00790090000D12055C7C
:100FE000E075F003A424D6F582E43401F583EBF038
:100FF000A3EAF0A3E9F0D2AF90000312055CE0FF92
:061000008004D2AF7F283E
:0610060090000E02053807
:1017620090FFFE120538EEF0A3EFF085088385099D
:1017720082E0FEA3E0FFD39400EE9400405FC2AF8C
:10178200780D860308E6FA08E6F990000E12013594
:101792002469F582E43402F583C083C082E0FD78D7
:1017A2000D860308E6FA08E6F990000F120135F4F7
:1017B200FCED5CD082D083F0700B900010120135EA
:1017C200F4780A56F6780D860308E6FA08E6F990E8
:1017D2000009EE8FF012029CD2AF12153790000270
:0317E200020538C5
:100CC00090FFFF120538EBF090FFFF120538EDF0B2
:0E0CD00090FFFF120538EFF090FFFA12053882
:100CDE0090000612055CE0D39400502D9000071290
:100CEE00055CE0D39400502190000812055CE0D31F
:100CFE009400501590000912055CE0FEA3E0D39419
:100D0E0000EE94005003020E8490000712055CE082
:100D1E00FED3943B40057F51020E869000081205CB
:100D2E005CE0D3943B40057F52020E869000091280
:100D3E00055CE0FCA3E0D394E7EC940340057F53FD
:100D4E00020E86AF06E4FCFDFE7B3CFAF9F81202B9
:100D5E00C9C004C005C006C00790000612055CE0BD
:100D6E00FFE4FCFDFE7B107A0EF9F81202C9D003E7
:100D7E00D002D001D000EF2BFBEE3AFAED39F9ECB0
:100D8E0038F890000812055CE0FFE4FCFDFEEB2F46
:100D9E00FFEE3AFEED39FDEC38FCE47B32FAF9F861
:100DAE001202C9C004C005C006C007900009120592
:100DBE005CE0FEA3E0FFEF240AFFE43EFEE433FD19
:100DCE00E433FCE47B32FAF9F81202C9E47BE87AE8
:100DDE0003F9F8120354D003D002D001D000EB2F48
:100DEE00FFEA3EFEE93DFDE83CFC8508838509826D
:100DFE001203FEE4FBFA7901F8850883850982E087
:100E0E00FCA3E0FDA3E0FEA3E0FF12035490000458
:100E1E0012055CEEF0A3EFF0850883850982C0838E
:100E2E00C082A3A3E0FEA3E0FFE4FDFCD082D0834A
:100E3E001203FE850883850982A3A3E0FEA3E0FFCB
:100E4E0012176290000412055CE0FEA3E0D394003A
:100E5E00EE9400401D7E807F001217627E807F0020
:100E6E0012176290000412055C74FFF5F01201EB8C
:080E7E0080D17F0080027F5447
:060E860090000B0205388C
:061B000090FFFC12053805
:101B0600C2AF9001D2E0FCA3E0FDA3E0FEA3E0FF9C
:101B16008508838509821203FED2AF85088385096D
:0C1B260082E0FCA3E0FDA3E0FEA3E0FFD2
:061B3200900004020538DA
:101B960090FFFC1205381203FEC2AF850883850943
:101BA60082E0FCA3E0FDA3E0FEA3E0FF9001D212D9
:0A1BB60003FED2AF900004020538D0
:030000000214A542
:1014A500787FE4F6D8FD75088075090075811F02FF
:0214B50014F22F
:101A210012000A780D088683088682A3E0F8A3E0F5
:101A3100F988838982E0FD7820A308E0F6DDFA8841
:101A410081A3E0F508A3E0F509780B7601D0E0FF6A
:101A5100D0E0FED0E0FDD0E0FCD0E0FBD0E0FAD059
:101A6100E0F9D0E0F8D0D0D082D083D0F0D0E0D26D
:021A7100AF3292
:1019BB00C0E0C0F0C083C082C0D0E8C0E0E9C0E0A6
:1019CB00EAC0E0EBC0E0ECC0E0EDC0E0EEC0E0EF61
:1019DB00C0E0E581C39420FD780D088683088682DC
:1019EB00A3E0F8A3E0F988838982EDF07820A308BF
:1019FB00E6F0DDFAA3E508F0A3E509F012000A789A
:101A0B000D7911E7F60809E7F60809E7F6781E796C
:061A1B001FE7F6021A2489
:0A1BE400E581C39404F5810219DDC8
:1014B7000213EEE493A3F8E493A34003F68001F24A
:1014C70008DFF48029E493A3F85407240CC8C33336
:1014D700C4540F4420C8834004F456800146F6DF05
:1014E700E4800B010204081020408090111EE47E66
:1014F700019360BCA3FF543F30E509541FFEE493FA
:10150700A360010ECF54C025E060A840B8E493A3C0
:10151700FAE493A3F8E493A3C8C582C8CAC583CAEB
:10152700F0A3C8C582C8CAC583CADFE9DEE780BEA3
:01122D0000C0
:10002600E709F608DFFA8046E709F208DFFA803EBC
:1000360088828C83E709F0A3DFFA8032E309F608A9
:10004600DFFA8078E309F208DFFA807088828C8311
:10005600E309F0A3DFFA806489828A83E0A3F608C5
:10006600DFFA805889828A83E0A3F208DFFA804C9F
:1000760080D280FA80C680D4806980F28033801076
:1000860080A680EA809A80A880DA80E280CA8033DF
:1000960089828A83ECFAE493A3C8C582C8CCC58357
:1000A600CCF0A3C8C582C8CCC583CCDFE9DEE78027
:1000B6000D89828A83E493A3F608DFF9ECFAA9F0A6
:1000C600EDFB2289828A83ECFAE0A3C8C582C8CCFC
:1000D600C583CCF0A3C8C582C8CCC583CCDFEADE15
:1000E600E880DB89828A83E493A3F208DFF980CC77
:1000F60088F0EF60010E4E60C388F0ED2402B40470
:100106000050B9F582EB2402B4040050AF23234516
:06011600822390007673C5
:10011C00BB010689828A83E0225002E722BBFE02E1
:09012C00E32289828A83E4932214
:10013500BB010CE58229F582E5833AF583E022507F
:1001450006E92582F8E622BBFE06E92582F8E222C9
:0D015500E58229F582E5833AF583E49322E3
:10016200BB010689828A83F0225002F722BBFE017C
:02017200F32276
:10017400F8BB010DE58229F582E5833AF583E8F0C1
:10018400225006E92582C8F622BBFE05E92582C86D
:02019400F22255
:10019600BC000BBE0029EF8DF084FFADF022E4CC4D
:1001A600F875F008EF2FFFEE33FEEC33FCEE9DEC16
:1001B600984005FCEE9DFE0FD5F0E9E4CEFD22ED5C
:1001C600F8F5F0EE8420D21CFEADF075F008EF2FA6
:1001D600FFED33FD4007985006D5F0F222C398FD97
:0501E6000FD5F0EA2234
:1001EB00C5F0F8A3E028F0C5F0F8E582158270029F
:0601FB001583E038F0223C
:10020100A3F8E0C5F025F0F0E582158270021583B0
:06021100E0C838F0E8220D
:10021700BB0110E58229F582E5833AF583E0F5F025
:10022700A3E0225009E92582F886F008E622BBFE02
:100237000AE92582F8E2F5F008E222E5832AF58348
:08024700E993F5F0A3E993220D
:10024F00BB010DC58229C582C5833AC5830201EB67
:10025F005011C58229F808E5F026F618F5F0E58269
:10026F0036F622BBFE11C58229F808E225F0F5F01B
:10027F00F218E23582F222F8E58229F582E5832A27
:0D028F00F58374019325F0F5F0E493382217
:10029C00F8BB0111E58229F582E5833AF583E8F094
:1002AC00E5F0A3F0225009E92582C8F608A6F02251
:0D02BC00BBFE09E92582C8F2E5F008F22238
:1002C900E88FF0A4CC8BF0A42CFCE98EF0A42CFCD4
:1002D9008AF0EDA42CFCEA8EF0A4CDA8F08BF0A452
:1002E9002DCC3825F0FDE98FF0A42CCD35F0FCEBB1
:1002F9008EF0A4FEA9F0EB8FF0A4CFC5F02ECD3976
:0F030900FEE43CFCEAA42DCE35F0FDE43CFC22E2
:1003180075F008758200EF2FFFEE33FECD33CDCC9C
:1003280033CCC58233C5829BED9AEC99E58298401F
:100338000CF582EE9BFEED9AFDEC99FC0FD5F0D6FC
:10034800E4CEFBE4CDFAE4CCF9A88222B800C1B926
:100358000059BA002DEC8BF084CFCECDFCE5F0CB64
:10036800F97818EF2FFFEE33FEED33FDEC33FCEB9D
:1003780033FB10D703994004EB99FB0FD8E5E4F958
:10038800FA227818EF2FFFEE33FEED33FDEC33FC45
:10039800C933C910D7059BE99A4007EC9BFCE99A39
:1003A800F90FD8E0E4C9FAE4CCFB2275F010EF2F7E
:1003B800FFEE33FEED33FDCC33CCC833C810D7077E
:1003C8009BEC9AE899400AED9BFDEC9AFCE899F8B9
:0E03D8000FD5F0DAE4CDFBE4CCFAE4C8F9224C
:0C03E600E6FC08E6FD08E6FE08E6FF2243
:0C03F200ECF608EDF608EEF608EFF62237
:0C03FE00ECF0A3EDF0A3EEF0A3EFF02272
:10040A00D083D082E493F608740193F608740293B9
:09041A00F608740393F6740473F0
:10042300A8828583F0D083D08212043A12043A1250
:10043300043A12043AE473E493A3C583C5F0C58375
:10044300C8C582C8F0A3C583C5F0C583C8C582C823
:010453002286
:0C045400A42582F582E5F03583F58322B3
:10046000BB011A89828A83D0F0D0E0F8D0E0F9D0BD
:10047000E0FAD0E0FBE8C0E0C0F00205845016E9E5
:10048000F8D083D082D0E0F9D0E0FAD0E0FBC0828F
:10049000C083020572BBFE16E9F8D083D082D0E09B
:0F04A000F9D0E0FAD0E0FBC082C08302059622BB
:1004AF00BB010DE58229F582E5833AF58302057BD1
:1004BF005007E92582F8020569BBFE07E92582F896
:1004CF0002058DE58229F582E5833AF58302059FC2
:1004DF00BB0120E58229F582E5833AF583D0F0D080
:1004EF00E0F8D0E0F9D0E0FAD0E0FBE8C0E0C0F0EF
:1004FF000205845018E92582F8D083D082D0E0F924
:10050F00D0E0FAD0E0FBC082C083020572BBFE18B8
:10051F00E92582F8D083D082D0E0F9D0E0FAD0E09C
:09052F00FBC082C0830205962284
:10053800E5092582F582E5083583F583B508048544
:1005480082092210AF06858209F50822858209F5FD
:0405580008D2AF22F4
:0D055C00E5092582F582E5083583F5832247
:09056900E6FB08E6FA08E6F922B7
:09057200EBF608EAF608E9F622AE
:09057B00E0FBA3E0FAA3E0F92281
:09058400EBF0A3EAF0A3E9F02278
:09058D00E2FB08E2FA08E2F9229F
:09059600EBF208EAF208E9F22296
:0C059F00E493FB740193FA740293F922B8
:00000001FF
